:1000000000308A00E6280000831A0A28A500030EA3
:10001000A6000F288312A500030EA600A6140A0846
:10002000AD008A018313A50E0408A7002008A800CC
:100030002108A9002208AA002308AB002408AC006C
:1000400083128B1E25280B194F28270884002808A7
:10005000A0002908A1002A08A2002B08A3002C0850
:10006000A4002D088A00260E83008312250EA618F0
:10007000831609004A08A1014902031842284908C9
:10008000A0004E28A0010830CB00C90DA00D4A08E1
:1000900020020318A000A10DCB0B45287A289C3024
:1000A0008100BE1F5628B71F5F285828B71B63283A
:1000B000B708031D5F2836083E0203186328C014E2
:1000C0004008850067283530C005400885003F0896
:1000D0003E02031870283130C0044008850074289F
:1000E0000E30C00540088500BE0A3E08C9006330D6
:1000F000CA003A282008BE000B118A112528423078
:1001000084000008031991280230A100A001A00B6F
:100110008728A10B86289730A000A00B8D28800B84
:10012000842800341030A000A301C801C50CC40C01
:10013000031CA0284608A3070318C80A4708C807D5
:10014000C80CA30CA20CA10CA00B962800344308E9
:1001500045068039C700C31FB228C209C309C20AB5
:100160000319C30AC51FB928C409C509C40A03195C
:10017000C50AA101A201A001A3014508031DC328CE
:1001800044080319DD281030C6000310C20DC30D4A
:10019000A00DA30D45082302031DD028440820020A
:1001A000031CD9284408A002031CA3034508A3028A
:1001B0000314A10DA20DC60BC5280000C71FE5281A
:1001C000A109A209A10A0319A20AB32A84011F30B6
:1001D00083051F1383161F149F141F159F150730C7
:1001E00083129F00703083168F0070308F000730AD
:1001F000831299008316050806308312A000A00B15
:10020000FF28000019088C118316051183120511AF
:100210000C3095001F1383161F109F101F119F1184
:100220000108C03901388100F630831281000030A6
:10023000A10005389200FF308316920083128B16BE
:10024000C0308B0408306500BF01A3013F08B60031
:100250002308B7003608BE00AF01AE01BB01BA01EA
:10026000C001C10141081D3C031C4129851D3F29D6
:100270004230A000A00B3A290000C10A4029C10168
:100280003229851941298B12B901B80185195329E1
:100290000330A000A00B4A29000000000130B8077D
:1002A0000318B90A4629851D60290330A000A00B58
:1002B0005729000000000130B8070318B90A532974
:1002C000B301B20185196F290330A000A00B662984
:1002D000000000000130B2070318B30A6229851D2F
:1002E0007C290330A000A00B73290000000001301E
:1002F000B2070318B30A6F29AF01AE0185198B2924
:100300000330A000A00B8229000000000130AE07DE
:100310000318AF0A7E29851D98290330A000A00B81
:100320008F29000000000130AE070318AF0A8B29A7
:10033000B101B0018519A7290330A000A00B9E29A7
:10034000000000000130B0070318B10A9A29851D8A
:10035000B4290330A000A00BAB290000000001303D
:10036000B0070318B10AA7298B16B91BC529B9080C
:10037000031DBE293808B43C0318C5296430C200E7
:100380007F200230BA070318BB0AB91BCE29B9086F
:10039000031DD7293808813C031CD7296430C200CB
:1003A0007F200230BA020030031C0130BB02B31BB5
:1003B000E029B308031DE3293208683C031CE32944
:1003C000B3016430B200B31BEF29B308031DEC295D
:1003D0003208B43C0318EF29B301CD30B200B31B8F
:1003E0000C2AB308031DF8293208A03C03180C2A74
:1003F0009B303202C2003308C3000030031C0130BE
:10040000C3024308C5004208C400C7010230C60049
:1004100092202108BF000D2ABF012F08B5002E0829
:10042000B400AF1B1A2AAF08031D1D2A2E086D3C0D
:10043000031C1D2AAF01AE01402AAF1B2B2AAF08B7
:10044000031D262A2E08BE3C03182B2A0330AF00BA
:10045000FF30AE00402A64302E02C2002F08C300D5
:100460000030031C0130C3024308C5004208C40029
:10047000C7010A30C60092202208AF002108AE0052
:100480002F08A2002E08A100A20CA10CA20CA10C06
:10049000A20C21089300A20C220C3039A0001508F0
:1004A000CF39200495006430B4020030031C0130C1
:1004B000B502B11B622AB108031D652A30086D3CE4
:1004C000031C652AB1016430B000B11B712AB10868
:1004D000031D6E2A3008C83C0318712AB101C830C8
:1004E000B000B11B862AB108031D7A2A3008953C5A
:1004F0000318862AB11B832AB108031D862A3008F7
:10050000A03C031C862AB1019B30B000B51B8F2A8A
:10051000B508031DAB2A34082C3C031CAB2A9B30C6
:100520003002A0003108A3000030031C0130A302F8
:1005300020083407C2003508C3000318C30A230883
:10054000C3073A084207B6004308B7000318B70AC2
:100550003B08B707E12A3508C3003408C200C501CB
:100560000A30C400A7282208C3002108C2002208BC
:10057000C5002108C400C7010730C60092200E3014
:100580002107C5002208C6000318C60A9B303002A6
:10059000A0003108A3000030031C0130A302200892
:1005A0004507C7004608C8000318C80A2308C8073B
:1005B0003A084707B6004808B7000318B70A3B08CF
:0605C000B70731296300BA
:02400E00C43CB0
:00000001FF
